:020000040800F2
:10000000101A00208901000835420008E53F000869
:100010003142000815030008B96300080000000021
:10002000000000000000000000000000055F000864
:100030001105000800000000554D00085D5F000834
:10004000A3010008A3010008A3010008A301000800
:10005000A3010008A3010008A3010008A3010008F0
:10006000A3010008A3010008A3010008A3010008E0
:10007000A3010008A3010008A3010008A3010008D0
:10008000A3010008A3010008A30100089963000868
:10009000A96300081903000829030008A301000848
:1000A000A3010008A3010008A3010008A3010008A0
:1000B000A3010008A301000805600008A3010008CF
:1000C000A3010008A3010008A3010008A301000880
:1000D000A3010008A3010008A3010008A301000870
:1000E000A3010008A3010008A301000800F002F822
:1000F00000F03AF80AA090E8000C82448344AAF188
:100100000107DA4501D100F02FF8AFF2090EBAE885
:100110000F0013F0010F18BFFB1A43F0010318473B
:10012000C0640000E0640000103A24BF78C878C1C1
:10013000FAD8520724BF30C830C144BF04680C60ED
:10014000704700000023002400250026103A28BF35
:1001500078C1FBD8520728BF30C148BF0B60704739
:100160001FB51FBD10B510BD00F08AF81146FFF78E
:10017000F7FF06F0B3F900F0A8F803B4FFF7F2FFB9
:1001800003BC00F0AFF80000094880470948004769
:10019000FEE7FEE7FEE7FEE7FEE7FEE7FEE7FEE737
:1001A000FEE7FEE704480549054A064B7047000094
:1001B00001600008ED00000810140020101A002053
:1001C000101600201016002010B5203AC0F00B8049
:1001D000B1E81850A0E81850B1E81850A0E818503D
:1001E000203ABFF4F5AF5FEA027C24BFB1E81850B3
:1001F000A0E8185044BF18C918C0BDE810405FEA15
:10020000827C24BF51F8043B40F8043B08BF704790
:10021000D20728BF31F8023B48BF11F8012B28BF95
:1002200020F8023B48BF00F8012B70474FF0000256
:1002300000B5134694469646203922BFA0E80C50DC
:10024000A0E80C50B1F12001BFF4F7AF090728BFB7
:10025000A0E80C5048BF0CC05DF804EB890028BF33
:1002600040F8042B08BF704748BF20F8022B11F05C
:10027000804F18BF00F8012B7047704770477047D8
:10028000754600F02BF8AE4605006946534620F04F
:100290000700854618B020B5FFF784FFBDE8204071
:1002A0004FF000064FF000074FF000084FF0000B32
:1002B000AC46ACE8C009ACE8C009ACE8C009ACE8A1
:1002C000C00921F007018D46704710B50446AFF311
:1002D00000802046BDE81040FFF74FBF0048704740
:1002E0001000002001491820ABBEFEE726000200E6
:1002F0007047000040F6CC00C2F20000007840F2E7
:100300000001C2F200010978401A813000F07F003C
:1003100070470000FFE7FEE780B540F6E000C2F25C
:10032000000000F06DFC80BD80B540F6E000C2F238
:10033000000000F065FC80BD40F27001C2F20001D7
:10034000486901304861704740F27001C2F2000113
:10035000C8690130C861704740F27001C2F2000103
:10036000886801308860704740F27001C2F2000175
:10037000886901308861704740F27001C2F2000163
:10038000086A01300862704740F27001C2F2000151
:10039000486801304860704740F27001C2F20001C5
:1003A000086801300860704740F27001C2F2000135
:1003B000086901300861704740F27001C2F2000123
:1003C000886C01308864704740F27001C2F200010D
:1003D000C86C0130C864704740F27001C2F200017D
:1003E000086D01300865704740F27001C2F20001EB
:1003F000486D01304865704740F27001C2F200015B
:10040000486A01304862704740F27001C2F2000150
:10041000886A01308862704740F27001C2F20001C0
:10042000C8680130C860704740F27001C2F2000134
:10043000486C01304864704740F27001C2F200011C
:10044000C86A0130C862704740F27001C2F2000110
:10045000486B01304863704740F27001C2F20001FE
:10046000C86B0130C863704740F27001C2F20001EE
:10047000086B01300863704740F27001C2F200015E
:10048000886B01308863704740F27001C2F200014E
:10049000086C01300864704780B590B0DDF848C042
:1004A000CDF83CC00E930D920C910B90002004905F
:1004B000042107918DF8280008900C9A019962F3A5
:1004C0001C0101919DF8071041F008018DF80710FB
:1004D0009DF8061001F0F00108318DF80610FF219B
:1004E0008DF800108DF801000099ADF80410019905
:1004F00021F060410691099040F6D400C2F200005C
:10050000006805A902AA04AB00F036F810B080BD5F
:100510007047000081B0EFF3108072B60090FFE7E3
:10052000FEE7000084B002900191029890F820004C
:100530008DF803009DF80300012805D0FFE79DF822
:10054000030002280AD1FFE7019A0298016848696E
:100550001043486100208DF80F0008E00299486AB6
:1005600040F48020486201208DF80F00FFE79DF8DD
:100570000F0004B07047000088B006900591049207
:100580000393069890F820008DF8070006980068FD
:10059000806800900598806808B9FFE700E0FFE7F1
:1005A0009DF80700012806D0FFE79DF80700022804
:1005B00040F08080FFE79DF80300400700280CD43E
:1005C000FFE79DF803000007002806D4FFE79DF829
:1005D0000300C006002864D5FFE70098C0F301605F
:1005E000029002990120884003990860059880686C
:1005F00068B9FFE705980168C06840EA415006996C
:100600000968029A01EB0211C1F880010EE0059918
:100610004A688868C96840EAC200084306990968C0
:10062000029A01EB0211C1F88001FFE70598006909
:1006300006990968029A01EB0211C1F88401059834
:10064000007D01280CD1FFE706980068029900EBB5
:100650000111D1F8840140F48070C1F88401FFE7F2
:100660000498406806990968029A01EB0211C1F8E2
:100670008C010498006806990968029A01EB02113E
:10068000C1F8880106980068029900EB0111D1F8C1
:10069000800140F00100C1F8800100208DF81F00AA
:1006A00011E00699486A40F40010486201208DF874
:1006B0001F0008E00699486A40F480204862012043
:1006C0008DF81F00FFE79DF81F0008B0704700007D
:1006D00086B004900391049800680190049890F803
:1006E00020008DF803009DF80300012806D0FFE7E5
:1006F0009DF80300022840F09B80FFE70199D1F8A4
:10070000000240F00100C1F800020398406900F0C7
:100710001F01012088400290029A0199D1F81C0221
:100720009043C1F81C020398C069F0B9FFE7029A30
:100730000199D1F80C029043C1F80C02039A9088F9
:10074000D168526940EA0140019901EBC201C1F848
:100750004002039A10889168526940EA0140019969
:1007600001EBC201C1F84402FFE70398C069012808
:100770001ED1FFE7029A0199D1F80C021043C1F88B
:100780000C02039A90881168526940EA014001996D
:1007900001EBC201C1F84002039A90899168526945
:1007A00040EA0140019901EBC201C1F84402FFE7B0
:1007B0000398806940B9FFE7029A0199D1F80402D1
:1007C0009043C1F8040207E0029A0199D1F80402AB
:1007D0001043C1F80402FFE70398006940B9FFE73E
:1007E000029A0199D1F814029043C1F8140207E06B
:1007F000029A0199D1F814021043C1F81402FFE7DC
:100800000398006A012808D1FFE7029A0199D1F8FC
:100810001C021043C1F81C02FFE70199D1F8000245
:1008200020F00100C1F8000200208DF8170008E058
:100830000499486A40F48020486201208DF817002E
:10084000FFE79DF8170006B07047000080B582B042
:1008500001900198406A08B9FFE7C4E00198406A36
:10086000C00718B1FFE7FFF797FDFFE70198406A5F
:100870008007002803D5FFE7FFF786FDFFE7019813
:10088000406A4007002803D5FFE7FFF765FDFFE753
:100890000198406A0007002803D5FFE7FFF7BCFD79
:1008A000FFE70198406AC006002803D5FFE7FFF77D
:1008B0007BFDFFE70198406A8006002803D5FFE72B
:1008C000FFF73AFDFFE70198406A4006002803D58C
:1008D000FFE7FFF749FDFFE70198406A000600289F
:1008E00003D5FFE7FFF730FDFFE70198406AC00539
:1008F000002803D5FFE7FFF73FFDFFE70198406AB7
:100900008005002803D5FFE7FFF776FDFFE7019894
:10091000406A4005002803D5FFE7FFF775FDFFE7B4
:100920000198406A0005002803D5FFE7FFF784FD22
:10093000FFE70198406AC004002803D5FFE7FFF7EE
:1009400093FDFFE70198406A8004002803D5FFE784
:10095000FFF77AFDFFE70198406A4004002803D5BD
:10096000FFE7FFF789FDFFE70198406A00040028D0
:1009700003D5FFE7FFF770FDFFE70198406AC0036A
:10098000002803D5FFE7FFF77FFDFFE70198406AE6
:100990008003002803D5FFE7FFF746FDFFE7019836
:1009A000406A4003002803D5FFE7FFF705FDFFE796
:1009B0000198406A0003002803D5FFE7FFF704FD14
:1009C000FFE70198406AC002002803D5FFE7FFF760
:1009D00003FDFFE70198406A8002002803D5FFE786
:1009E000FFF702FDFFE702B080BD000086B0049073
:1009F000039102920193049890F820008DF803006F
:100A00009DF80300012806D0FFE79DF803000228A7
:100A100040F0E880FFE7039880B9FFE7049800689A
:100A2000C068800748B9FFE70499486A40F400109D
:100A3000486201208DF81700DDE00FE0049800689F
:100A40000069800748B9FFE70499486A40F400103C
:100A5000486201208DF81700CDE0FFE70498006898
:100A6000039900EB0110D0F8B00100F004000299E6
:100A700088600298806858B9FFE704980068039975
:100A800000EB0110D0F8B001400D029908600AE0B7
:100A900004980068039900EB0110D0F8B001C00879
:100AA00002994860FFE704980068039900EB011081
:100AB000D0F8B00100F002000299C8600498006804
:100AC000039900EB0110D0F8B40100F00F000828E2
:100AD00004D3FFE70299082008610BE0049800683E
:100AE000039900EB0110D0F8B40100F00F00029957
:100AF0000861FFE704980068039900EB0110D0F843
:100B0000B40180B2000A02998861049800680399D0
:100B100000EB0110D0F8B401000C02994861049870
:100B20000068039900EB0110D0F8B8010199087032
:100B300004980068039900EB0110D0F8B801000A8E
:100B40000199487004980068039900EB0110D0F8EF
:100B5000B801000C0199887004980068039900EBB3
:100B60000110D0F8B801000E0199C870049800680F
:100B7000039900EB0110D0F8BC01019908710498A9
:100B80000068039900EB0110D0F8BC01000A01993C
:100B9000487104980068039900EB0110D0F8BC017B
:100BA000000C0199887104980068039900EB01100A
:100BB000D0F8BC01000E0199C871039838B9FFE75D
:100BC00004980168C86840F02000C86006E00498F6
:100BD0000168086940F020000861FFE700208DF8F7
:100BE000170008E00499486A40F480204862012018
:100BF0008DF81700FFE79DF8170006B0704700005A
:100C000080B58AB009900020089009980068406972
:100C10000790099800684068069009980068806805
:100C2000059009980068C0680490099800680069F8
:100C3000039009980068806902909DF81C00C00725
:100C4000002800F09480FFE79DF81400C00758B317
:100C5000FFE709980168012088609DF8140080076B
:100C6000002804D5FFE70998816A88471BE09DF8B2
:100C700014004007002805D5FFE7089840F40060FD
:100C800008900FE09DF814000007002805D5FFE745
:100C9000089840F48050089003E00998416B884719
:100CA000FFE7FFE7FFE7FFE79DF81500C00760B328
:100CB000FFE7099801684FF4807088609DF815007F
:100CC0008007002804D5FFE70998C16A88471BE020
:100CD0009DF815004007002805D5FFE7089840F467
:100CE000005008900FE09DF815000007002805D57A
:100CF000FFE7089840F48040089003E00998816B72
:100D00008847FFE7FFE7FFE7FFE79DF81600C0070A
:100D100060B3FFE7099801684FF4803088609DF860
:100D200016008007002804D5FFE70998016B884763
:100D30001BE09DF816004007002805D5FFE708983E
:100D400040F4004008900FE09DF8160000070028CE
:100D500005D5FFE7089840F48030089003E0099833
:100D6000C16B8847FFE7FFE7FFE7FFE7FFE79DF875
:100D70001C000007002810D5FFE79DF81000C006F2
:100D8000002809D5FFE7089840F4007008900998FA
:100D900001681020C860FFE7FFE79DF81C004007CE
:100DA00000280FD5FFE79DF810000007002808D5A0
:100DB000FFE7099801680820C8600998416C8847D6
:100DC000FFE7FFE79DF81C00800700280BD5FFE731
:100DD00009980068C068800720B1FFE70998016C96
:100DE0008847FFE7FFE79DF81C004006002810D564
:100DF000FFE79DF80C00C006002809D5FFE708981A
:100E000040F4806008900998016810200861FFE7AD
:100E1000FFE79DF81C00800600280FD5FFE79DF82E
:100E20000C000007002808D5FFE709980168082092
:100E300008610998C16C8847FFE7FFE79DF81C002F
:100E4000C00600280BD5FFE70998006800698007F5
:100E500020B1FFE70998816C8847FFE7FFE79DF81D
:100E60001E00800700280FD5FFE79DF81800C00678
:100E7000002808D5FFE70998016810204860099804
:100E8000016D8847FFE7FFE79DF81E00C00778B1B6
:100E9000FFE79DF818000007002808D5FFE709982C
:100EA0000168082048600998416D8847FFE7FFE71F
:100EB0009DF81D000006002840F18D80FFE79DF899
:100EC00018004007002840F18180FFE79DF81D00D1
:100ED000C00750B1FFE79DF80800C00728B1FFE741
:100EE000089840F001000890FFE79DF81D0080077A
:100EF00000280BD5FFE79DF808008007002805D5DE
:100F0000FFE7089840F002000890FFE79DF81D00F9
:100F1000400700280BD5FFE79DF808004007002890
:100F200005D5FFE7089840F004000890FFE79DF81A
:100F30001D000007002848D5FFE79DF8080010F0C5
:100F4000700F42D0FFE7029800F070000146019157
:100F5000102814D0FFE70198202815D0FFE701984A
:100F6000302816D0FFE70198402817D0FFE70198F6
:100F7000502818D0FFE70198602819D01DE0089884
:100F800040F00800089019E0089840F01000089020
:100F900014E0089840F0200008900FE0089840F016
:100FA000400008900AE0089840F08000089005E0B2
:100FB000089840F48070089000E0FFE70998016805
:100FC000886920F070008861FFE7FFE709980168F1
:100FD00004204860FFE7089848B1FFE7089A09999C
:100FE000486A104348620998816D8847FFE70AB054
:100FF00080BD000080B584B00290029820B9FFE760
:1010000001208DF80F003AE1029890F820000028A6
:101010005DD1FFE7029941F24D50C0F6000008642F
:10102000029941F24550C0F600004864029941F22D
:101030005D50C0F600008864029941F25550C0F638
:101040000000C864029941F20160C0F600008862A5
:10105000029941F21160C0F60000C862029941F2A3
:101060002160C0F600000863029941F2F950C0F611
:1010700000004863029941F20960C0F600008863ED
:10108000029941F21960C0F60000C863029941F26A
:101090006550C0F600000865029941F2F170C0F693
:1010A00000004865029940F64D00C0F600008865D2
:1010B0000298C06D38B9FFE7029941F2E120C0F60D
:1010C0000000C865FFE70298C16D8847FFE70298F6
:1010D0000168086840F00100086000F0EDFD019033
:1010E000FFE7029800684068C007A8B9FFE700F072
:1010F000E3FD0199401A0B280DD3FFE70299486AD6
:1011000040F4003048620299052081F82000012057
:101110008DF80F00B3E0E4E702980168086820F05A
:101120000200086000F0C8FD0190FFE70298006827
:1011300040688007002815D5FFE700F0BDFD019944
:10114000401A0B280DD3FFE70299486A40F400309B
:1011500048620299052081F8200001208DF80F00D7
:101160008DE0E3E70298007E012807D1FFE70298AF
:101170000168086840F08000086006E00298016895
:10118000086820F080000860FFE70298407E012890
:1011900007D1FFE702980168086840F04000086046
:1011A00006E002980168086820F040000860FFE748
:1011B0000298807E012807D1FFE70298016808683D
:1011C00040F02000086006E002980168086820F0FE
:1011D00020000860FFE70298C07E012807D1FFE7E2
:1011E00002980168086820F01000086006E0029884
:1011F0000168086840F010000860FFE70298007F6F
:10120000012807D1FFE702980168086840F008004C
:10121000086006E002980168086820F0080008608D
:10122000FFE70298407F012807D1FFE70298016895
:10123000086840F00400086006E002980168086849
:1012400020F004000860FFE7029B19685A6898685C
:10125000D3F80CC040EA0C00D3F810C040EA0C00F0
:101260005B691843013A1043C86102990020486243
:10127000029A012182F820108DF80F00FFE79DF8F7
:101280000F0004B080BD000080B582B001900198CD
:10129000006846F20041C4F2000188421DD1FFE718
:1012A00041F21C01C4F20201086820F000700860DD
:1012B00040F60000C4F201004FF4C05100F09CFA67
:1012C000132000F07BFD142000F078FD152000F0C5
:1012D00075FD162000F072FDFFE702B080BD000032
:1012E00080B58EB00D9000200C900B900A90099064
:1012F0000D98006846F20041C4F2000188425ED1B8
:10130000FFE7FFE741F21C00C4F20200016841F070
:1013100000710160006800F0007008900898FFE715
:10132000FFE741F21800C4F20200016841F0040135
:101330000160006800F0040007900798FFE74FF491
:1013400000600990002005900A900B9040F6000084
:10135000C4F20100009009A9019100F01DFB009862
:1013600001994FF48052099202220A9203220C92B0
:1013700000F012FB059A13200290114600F032FD96
:10138000029800F025FD059A14200390114600F004
:1013900029FD039800F01CFD059A152004901146C4
:1013A00000F020FD049800F013FD059A1620069029
:1013B000114600F017FD069800F00AFDFFE70EB099
:1013C00080BD000087B005908DF8131003920020B7
:1013D0008DF80B00039848B9FFE70599486A40F477
:1013E0008000486201208DF81B00A6E0059890F867
:1013F0002000012870D1FFE79DF8130001460191FC
:101400000E285FD801990FF2080000EB8100874693
:1014100000F01CB800F01EB800F020B800F022B8B0
:1014200000F024B800F026B800F028B800F02AB880
:1014300000F02CB800F02EB800F030B800F032B850
:1014400000F034B800F036B800F038B803980599C9
:10145000886240E003980599C8623CE003980599CA
:10146000086338E003980599486334E003980599C8
:10147000886330E003980599C8632CE003980599C8
:10148000086428E003980599486424E003980599C6
:10149000886420E003980599C8641CE003980599C6
:1014A000086518E003980599486514E003980599C4
:1014B000886510E003980599C8650CE003980599C4
:1014C000086608E00599486A40F4800048620120F7
:1014D0008DF80B00FFE72BE0059890F82000E8B9A5
:1014E000FFE79DF81300014600910D2804D0FFE7A7
:1014F00000980E2804D007E003980599C8650CE011
:1015000003980599086608E00599486A40F4800048
:10151000486201208DF80B00FFE708E00599486A52
:1015200040F48000486201208DF80B00FFE7FFE7E0
:101530009DF80B008DF81B00FFE79DF81B0007B01E
:101540007047000081B0009001B0704781B00090FA
:1015500001B0704781B0009001B0704781B0009039
:1015600001B0704781B0009001B0704780B584B081
:101570000290029890F8200001282FD1FFE70299ED
:10158000022081F8200002980168086820F001001C
:10159000086000F091FB0190FFE702980068406846
:1015A000C007A8B1FFE700F087FB0199401A0B289C
:1015B0000DD3FFE70299486A40F40030486202996F
:1015C000052081F8200001208DF80F000FE0E4E7EE
:1015D0000299002048628DF80F0008E00299486ADD
:1015E00040F40020486201208DF80F00FFE79DF8CD
:1015F0000F0004B080BD000081B0009001B07047C2
:1016000081B0009001B0704781B0009001B0704788
:1016100081B0009001B0704781B0009001B0704778
:1016200081B0009001B0704784B003908DF80B102A
:1016300000208DF80A00039890F82000012840F05F
:10164000A080FFE79DF80B00014601910E2800F2F3
:101650008E8001990FF2080000EB8100874600BFE1
:1016600000F01CB800F021B800F026B800F02BB84C
:1016700000F030B800F035B800F03AB800F03FB8EC
:1016800000F044B800F049B800F04EB800F053B88C
:1016900000F058B800F05DB800F062B8039941F26C
:1016A0000160C0F6000088626AE0039941F21160AF
:1016B000C0F60000C86263E0039941F22160C0F601
:1016C000000008635CE0039941F2F950C0F60000A5
:1016D000486355E0039941F20960C0F60000886351
:1016E0004EE0039941F21960C0F60000C86347E07C
:1016F000039941F24D50C0F60000086440E00399A0
:1017000041F24550C0F60000486439E0039941F2C7
:101710005D50C0F60000886432E0039941F25550F4
:10172000C0F60000C8642BE0039941F26550C0F692
:101730000000086524E0039941F2F170C0F6000052
:1017400048651DE0039940F64D00C0F6000088652D
:1017500016E0039941F2E120C0F60000C8650FE0F1
:10176000039941F28920C0F60000086608E0039959
:10177000486A40F48000486201208DF80A00FFE7C3
:1017800031E0039890F8200018BBFFE79DF80B00AC
:10179000014600910D2804D0FFE700980E2807D0DD
:1017A0000DE0039941F2E120C0F60000C8650FE0AA
:1017B000039941F28920C0F60000086608E0039909
:1017C000486A40F48000486201208DF80A00FFE773
:1017D00008E00399486A40F48000486201208DF8CF
:1017E0000A00FFE7FFE79DF80A0004B07047000019
:1017F00081B0009001B070478DB00C900B9100202B
:101800000A90FFE70B980A99C840002800F0C180B1
:10181000FFE70B980A9A0121914008400990099826
:10182000002800F0B280FFE70A9820F003000821AA
:10183000C4F20101405808900A9800F003008100AA
:101840000F2000FA01F108980840089008980590C8
:101850000C9840F60001C4F20101884203D1FFE771
:101860000020049026E00C9840F60041C4F20101EB
:10187000884203D1FFE70120039018E00C9841F261
:101880000001C4F20101884203D1FFE70220029067
:101890000AE00C9941F20042C4F201020420914294
:1018A00008BF03200290FFE702980390FFE7039828
:1018B0000490FFE7059804990A9A02F00302920047
:1018C0009140884232D1FFE7099A40F20041C4F2C8
:1018D0000101086890430860099A40F20441C4F28B
:1018E0000101086890430860099A40F20C41C4F273
:1018F0000101086890430860099A40F20841C4F267
:1019000001010868904308600A9800F00300810014
:101910000F2088400890089B0A9820F003010822B5
:10192000C4F20102885898438850FFE70998FF28BD
:1019300003D8FFE70C98019003E00C980430019065
:10194000FFE7019807900998FF2804D8FFE70A9855
:101950008000009006E00A996FF01F0000EB810004
:101960000090FFE70098069007980068069A0F21FC
:101970009140884304219140084307990860099ADF
:101980000C99C8689043C860FFE70A9801300A9034
:1019900038E70DB07047000090B00F900E91002016
:1019A0000D900990FFE70E9800680D99C840002837
:1019B00000F07F81FFE70D99012088400C900E9880
:1019C00000680C9908400B900B980C99884240F0E5
:1019D0006C81FFE70E9840680590002851D0FFE722
:1019E000059801283AD0FFE7059802283FD0FFE785
:1019F000059803285FD0FFE70598112832D0FFE74C
:101A00000598122838D0FFE705980021C1F211018E
:101A1000884236D0FFE705980021C1F212018842C2
:101A20002FD0FFE705980021C1F22101884228D07C
:101A3000FFE705980021C1F22201884221D0FFE78B
:101A400005980021C1F2310188421AD0FFE70598BC
:101A50000021C1F23201884213D02FE00E98C068F5
:101A600009902CE00E98C0680430099027E00E9889
:101A7000C0680830099022E00E98C0680C300990C8
:101A80001DE00E98806818B9FFE70420099011E066
:101A90000E988068012806D1FFE7082009900C986D
:101AA0000F99086105E0082009900C980F9948618A
:101AB000FFE7FFE703E00020099000E0FFE70B9855
:101AC000FF2803D8FFE70F98049003E00F98043035
:101AD0000490FFE7049808900B98FF2804D8FFE7CC
:101AE0000D988000039006E00D996FF01F0000EB49
:101AF00081000390FFE70398079008980068079A11
:101B00000F21914088430999914008430899086042
:101B10000E98C079C006002840F1C680FFE7FFE7B5
:101B200041F21800C4F20200016841F001010160B5
:101B3000006800F0010006900698FFE70D9820F07D
:101B400003000821C4F2010140580A900D9800F0EA
:101B5000030081000F2000FA01F10A9888430A90DF
:101B60000F9840F60001C4F20101884203D1FFE75B
:101B70000020029026E00F9840F60041C4F20101D7
:101B8000884203D1FFE70120019018E00F9841F24D
:101B90000001C4F20101884203D1FFE70220009056
:101BA0000AE00F9941F20042C4F20102042091427E
:101BB00008BF03200090FFE700980190FFE701981D
:101BC0000290FFE702980D9901F00301890000FAE5
:101BD00001F10A9808430A900A980D9921F003012F
:101BE0000822C4F2010288500E988079C0060028AD
:101BF00009D5FFE70B9A40F20841C4F201010868D9
:101C00001043086008E00B9A40F20841C4F2010159
:101C1000086890430860FFE70E98807980060028E6
:101C200009D5FFE70B9A40F20C41C4F201010868A4
:101C30001043086008E00B9A40F20C41C4F2010125
:101C4000086890430860FFE70E98807980070028B5
:101C500009D5FFE70B9A40F20441C4F2010108687C
:101C60001043086008E00B9A40F20441C4F20101FD
:101C7000086890430860FFE70E988079C00748B174
:101C8000FFE70B9A40F20041C4F2010108681043DB
:101C9000086008E00B9A40F20041C4F201010868B4
:101CA00090430860FFE7FFE7FFE70D9801300D90D4
:101CB00079E610B07047000041F20C40C2F200001B
:101CC0000068704740F20800C2F20000027841F25A
:101CD0000C41C2F20001086810440860704700001F
:101CE00080B542F20001C4F20201086840F0100021
:101CF0000860032000F090F80F2000F005F800F0D5
:101D00003BF8002080BD000080B582B0009040F21A
:101D10000400C2F20000006840F20801C2F20001B3
:101D20000A784FF47A71B1FBF2F1B0FBF1F001F0F7
:101D3000BDFA20B1FFE701208DF8070018E00098F8
:101D40000F280DD8FFE700994FF0FF30002200F078
:101D500049F8009840F20C01C2F20001086003E06B
:101D600001208DF8070003E000208DF80700FFE751
:101D70009DF8070002B080BD82B0FFE741F2180075
:101D8000C4F20200016841F001010160006800F046
:101D9000010001900198FFE7FFE741F21C00C4F247
:101DA0000200016841F080510160006800F080503D
:101DB00000900098FFE702B07047000080B582B045
:101DC0008DF807009DF9070004F0F8FA02B080BD15
:101DD00080B582B08DF807009DF9070004F00AFB7A
:101DE00002B080BD80B586B08DF8170004910392D3
:101DF0000020029004F016FB02909DF9170001905C
:101E000002980499039A02F017FA0146019804F027
:101E100011FB06B080BD000080B582B00190019832
:101E200004F02AFB02B080BD2021C4F20E21012063
:101E30000860704780B588B0079000200690059034
:101E400004900390029007980190012866D0FFE764
:101E50000198022800F0A580FFE70198102840F0C3
:101E6000B080FFE741F20400C4F202000068039072
:101E700041F20000C4F202000068C00100284CD505
:101E8000FFE70398C0F3834146F2BC50C0F6000060
:101E9000405C04909DF80E00C007F0B1FFE741F2EE
:101EA0000400C4F202000068C0F3404146F2CC5086
:101EB000C0F60000405C06909DF80E00C00758B1C7
:101EC000FFE7069941F20020C0F27A00B0FBF1F082
:101ED000049948430590FFE707E0049840F6001195
:101EE000C0F23D0148430590FFE741F20400C4F20F
:101EF000020000684002002803D5FFE70598029021
:101F00000AE0059840004AF6AB21CAF6AA21A0FBD8
:101F1000011040080290FFE7FFE753E041F2200084
:101F2000C4F2020000680390039800F44070B0F51A
:101F3000807F0AD1FFE79DF80C008007002804D5B8
:101F4000FFE74FF4004002902AE0039800F440704D
:101F5000B0F5007F0DD1FFE741F22400C4F202008A
:101F600000688007002804D5FFE749F6404002904A
:101F700015E0039800F44070B0F5407F0DD1FFE705
:101F800041F20000C4F2020000688003002804D57A
:101F9000FFE74FF22440029000E0FFE7FFE7FFE792
:101FA00010E000F029FA41F20401C4F202010968CC
:101FB00001F44042022101EB5231B0FBF1F00290FA
:101FC00000E0FFE7029808B080BD000080B586B051
:101FD000049000200390029004980078C007002825
:101FE00000F0AC80FFE700208DF8070041F21C00F4
:101FF000C4F202000068C000002813D4FFE7FFE726
:1020000041F21C00C4F20200016841F080510160FD
:10201000006800F0805000900098FFE701208DF8E4
:102020000700FFE747F20000C4F200000068C005A7
:10203000002822D4FFE747F20001C4F2000108683B
:1020400040F480700860FFF737FE0390FFE747F227
:102050000000C4F200000068C00500280CD4FFE7AF
:10206000FFF72AFE0399401A652804D3FFE70320EF
:102070008DF817008AE0EAE7FFE741F22000C4F29A
:102080000200006800F4407002900298E0B3FFE79D
:1020900002980499496801F44071884234D0FFE7FE
:1020A00041F22001C4F20201086820F4407002905D
:1020B00040F24042C4F24222012010600020106031
:1020C000029808609DF80800C007E0B1FFE7FFF73D
:1020D000F3FD0390FFE741F22000C4F20200006824
:1020E000800700280ED4FFE7FFF7E6FD0399401AAA
:1020F00041F28931884204D3FFE703208DF81700AD
:1021000044E0E8E7FFE7FFE741F22001C4F2020103
:10211000086820F44070049A5268104308609DF8E3
:102120000700012809D1FFE741F21C01C4F20201B6
:10213000086820F080500860FFE7FFE70498007807
:10214000800700280CD5FFE741F20401C4F2020128
:10215000086820F44040049A926810430860FFE742
:1021600004980078C00600280CD5FFE741F204016E
:10217000C4F20201086820F48000049AD268104377
:102180000860FFE700208DF81700FFE79DF81700B3
:1021900006B080BD80B584B002900191029820B94C
:1021A000FFE701208DF80F001BE1019842F20001CA
:1021B000C4F20201096801F00701884216D9FFE75D
:1021C00042F20000C4F20200016821F00701019A06
:1021D00011430160006800F007000199884204D0B3
:1021E000FFE701208DF80F00FBE0FFE70298007881
:1021F000800700282AD5FFE70298007840070028CA
:1022000009D5FFE741F20401C4F20201086840F475
:10221000E0600860FFE7029800780007002809D511
:10222000FFE741F20401C4F20201086840F4605083
:102230000860FFE741F20401C4F20201086820F0DF
:10224000F000029A926810430860FFE70298007855
:10225000C007002860D0FFE70298406801280ED12F
:10226000FFE741F20000C4F202000068800300288A
:1022700004D4FFE701208DF80F00B2E021E00298BE
:10228000406802280ED1FFE741F20000C4F20200CC
:1022900000688001002804D4FFE701208DF80F00BA
:1022A0009FE00DE041F20000C4F2020000688007E8
:1022B000002804D4FFE701208DF80F0091E0FFE72C
:1022C000FFE741F20401C4F20201086820F00300B4
:1022D000029A526810430860FFF7EEFC0090FFE797
:1022E00041F20400C4F20200006800F00C00029900
:1022F0004968B0EB810F0ED0FFE7FFF7DDFC0099D6
:10230000401A41F28931884204D3FFE703208DF857
:102310000F0066E0E4E7FFE7019842F20001C4F233
:102320000201096801F00701884216D2FFE742F274
:102330000000C4F20200016821F00701019A114374
:102340000160006800F007000199884204D0FFE7AF
:1023500001208DF80F0044E0FFE702980078400765
:1023600000280CD5FFE741F20401C4F2020108681D
:1023700020F4E060029AD26810430860FFE70298F8
:102380000078000700280DD5FFE741F20401C4F2F0
:102390000201086820F46050029A126940EAC20003
:1023A0000860FFE700F03AF841F20401C4F20201CC
:1023B0000968C9B20A0946F2A451C0F60001895C55
:1023C000C84040F20401C2F20001086040F20C0073
:1023D000C2F200000068FFF797FC00208DF80F00A4
:1023E000FFE79DF80F0004B080BD000040F204003C
:1023F000C2F200000068704780B5FFF7F7FF41F2B6
:102400000401C4F202010968C1F3C22246F2B451C8
:10241000C0F60001895CC84080BD000086B0002085
:102420000590049003900290019041F20400C4F2E0
:10243000020000680590059800F00C00014600912C
:1024400000283FD0FFE70098042804D0FFE7009859
:10245000082806D037E041F20020C0F27A0001904F
:1024600037E00598C0F3834146F2CE50C0F6000035
:10247000405C02909DF81600C007C0B1FFE741F232
:102480000400C4F202000068C0F3404146F2DE508E
:10249000C0F60000405C0490029841F20021C0F2B6
:1024A0007A0148430499B0FBF1F0039007E00298E9
:1024B00040F60011C0F23D0148430390FFE7039846
:1024C000019006E0FFE741F20020C0F27A0001909F
:1024D000FFE7019806B0704780B588B00790069175
:1024E0000592002004900390029001900221029135
:1024F0000321049103904FF480700190FFE741F2B3
:102500001800C4F20200016841F004010160006893
:1025100000F0040000900098FFE740F60000C4F2CD
:10252000010001A9FFF738FA41F20401C4F20201E7
:10253000086820F0E060069A1043086008B080BD8B
:1025400080B586B00490049820B9FFE701208DF88B
:1025500017002EE304980078C007002800F0AE8032
:10256000FFE741F20400C4F20200006800F00C0032
:10257000042813D0FFE741F20400C4F2020000680F
:1025800000F00C0008281BD1FFE741F20400C4F260
:1025900002000068C003002812D5FFE741F20000E6
:1025A000C4F2020000688003002808D5FFE7049801
:1025B000406820B9FFE701208DF81700F9E27CE0C0
:1025C000FFE704984068B0F5803F09D1FFE741F28A
:1025D0000001C4F20201086840F48030086032E073
:1025E0000498406868B9FFE741F20001C4F20201B3
:1025F000086820F480300860086820F480200860B3
:1026000020E004984068B0F5A02F0DD1FFE741F21B
:102610000001C4F20201086840F4802008600868E4
:1026200040F4803008600CE041F20001C4F2020185
:10263000086820F480300860086820F48020086072
:10264000FFE7FFE7FFE7FFE704984068D0B1FFE747
:10265000FFF732FB0390FFE741F20000C4F20200F3
:102660000068800300280CD4FFE7FFF725FB0399DF
:10267000401A652804D3FFE703208DF8170098E27D
:10268000EAE719E0FFF718FB0390FFE741F20000CB
:10269000C4F202000068800300280CD5FFE7FFF7B2
:1026A0000BFB0399401A652804D3FFE703208DF83C
:1026B00017007EE2EAE7FFE7FFE7FFE7049800780C
:1026C0008007002840F18D80FFE741F20400C4F24A
:1026D0000200006810F00C0F13D0FFE741F2040075
:1026E000C4F20200006800F00C00082829D1FFE7BE
:1026F00041F20400C4F202000068C003002820D4A4
:10270000FFE741F20000C4F20200006880070028E1
:1027100009D5FFE704980069012804D0FFE70120EC
:102720008DF8170045E241F20001C4F20201086889
:1027300020F0F800049A526940EAC2000860FFE7FE
:102740004EE00498006958B3FFE70021C4F242212B
:1027500001200860FFF7B0FA0390FFE741F20000A4
:10276000C4F202000068800700280CD4FFE7FFF7DE
:10277000A3FA0399401A032804D3FFE703208DF836
:10278000170016E2EAE741F20001C4F2020108680C
:1027900020F0F800049A526940EAC20008601EE086
:1027A0000021C4F2422100200860FFF785FA03905F
:1027B000FFE741F20000C4F2020000688007002831
:1027C0000CD5FFE7FFF778FA0399401A032804D3E2
:1027D000FFE703208DF81700EBE1EAE7FFE7FFE7EB
:1027E000FFE7049800780007002848D5FFE7049821
:1027F000806918B3FFE740F28041C4F24221012012
:102800000860FFF759FA0390FFE741F22400C4F291
:1028100002000068800700280CD4FFE7FFF74CFA9D
:102820000399401A032804D3FFE703208DF817000B
:10283000BFE1EAE7012003F0B3F81FE040F2804176
:10284000C4F2422100200860FFF736FA0390FFE748
:1028500041F22400C4F202000068800700280CD571
:10286000FFE7FFF729FA0399401A032804D3FFE78B
:1028700003208DF817009CE1EAE7FFE7FFE70498E3
:1028800000784007002840F1D880FFE700208DF84D
:10289000070041F21C00C4F202000068C0000028DA
:1028A00013D4FFE7FFE741F21C00C4F20200016805
:1028B00041F080510160006800F080500090009865
:1028C000FFE701208DF80700FFE747F20000C4F2A0
:1028D00000000068C005002822D4FFE747F200018D
:1028E000C4F20001086840F480700860FFF7E4F962
:1028F0000390FFE747F20000C4F200000068C00543
:1029000000280CD4FFE7FFF7D7F90399401A652890
:1029100004D3FFE703208DF817004AE1EAE7FFE759
:10292000FFE70498C068012809D1FFE741F22001C0
:10293000C4F20201086840F00100086031E0049828
:10294000C06868B9FFE741F22001C4F202010868DB
:1029500020F001000860086820F0040008601FE013
:102960000498C06805280DD1FFE741F22001C4F2A8
:102970000201086840F004000860086840F00100A7
:1029800008600CE041F22001C4F20201086820F066
:1029900001000860086820F004000860FFE7FFE716
:1029A000FFE7FFE70498C068E0B1FFE7FFF784F9AD
:1029B0000390FFE741F22000C4F2020000688007A4
:1029C00000280ED4FFE7FFF777F90399401A41F288
:1029D0008931884204D3FFE703208DF81700E8E02F
:1029E000E8E71BE0FFF768F90390FFE741F22000FA
:1029F000C4F202000068800700280ED5FFE7FFF749
:102A00005BF90399401A41F28931884204D3FFE708
:102A100003208DF81700CCE0E8E7FFE79DF80700FA
:102A2000012809D1FFE741F21C01C4F20201086844
:102A300020F080500860FFE7FFE70498C069002895
:102A400000F0B380FFE741F20400C4F20200006826
:102A500000F00C00082800F08280FFE70498C069AD
:102A600002285CD1FFE76021C4F242210020086007
:102A7000FFF722F90390FFE741F20000C4F20200E1
:102A80000068800100280CD5FFE7FFF715F90399CE
:102A9000401A032804D3FFE703208DF8170088E0CD
:102AA000EAE70498006AB0F5803F0CD1FFE741F2F5
:102AB0000401C4F20201086820F40030049A92680C
:102AC00010430860FFE741F20401C4F20201086804
:102AD00020F47410049B1A6A5B6A1A43104308605E
:102AE0006021C4F2422101200860FFF7E5F803905D
:102AF000FFE741F20000C4F20200006880010028F4
:102B00000CD4FFE7FFF7D8F80399401A032804D341
:102B1000FFE703208DF817004BE0EAE71EE0602195
:102B2000C4F2422100200860FFF7C6F80390FFE7D7
:102B300041F20000C4F202000068800100280CD5B8
:102B4000FFE7FFF7B9F80399401A032804D3FFE71A
:102B500003208DF817002CE0EAE7FFE724E0049853
:102B6000C069012804D1FFE701208DF8170020E09B
:102B700041F20400C4F2020000680290029800F4DE
:102B800080300499096A884208D1FFE7029800F46E
:102B900070100499496A884204D0FFE701208DF83B
:102BA000170006E0FFE7FFE7FFE700208DF81700BA
:102BB000FFE79DF8170006B080BD000080B586B025
:102BC00004900391029200208DF80600ADF80400F5
:102BD000049818B1FFE7039820B9FFE701208DF8AA
:102BE000170034E0049801A9002200F035F820B164
:102BF000FFE701208DF8170029E00498007B039976
:102C000008700498C07B0399C8700498407B0399AE
:102C100048700498807B03998870029898B1FFE708
:102C20000398C07802F0F0FE0399C87003984078CA
:102C300002F0EAFE039948700398807802F0E4FEFF
:102C400003998870FFE700208DF81700FFE79DF8D3
:102C5000170006B080BD000080B588B006900591D1
:102C6000049200200390029001900090069818B101
:102C7000FFE7059820B9FFE701208DF81F00C0E0AD
:102C80000698006840684007002803D5FFE7012048
:102C900018B906E0012020B9FFE701208DF81F00D8
:102CA000AFE0069803F036F8039003994BF2C53075
:102CB000C9F2A210A1FB0021C90A0091039BA3FB4A
:102CC0000021C90A4FF4616201FB123348F6890101
:102CD000C8F68801A3FB01C35B09DDF814C08CF8BA
:102CE0000130039BA3FB00C0C00A00FB1230A0FB15
:102CF000011251090901A1EB5211A0EB81000599C4
:102D00008870009818285ED3FFE700984AF6AB2138
:102D1000CAF6AA21A0FB0120000901900098A0FB9F
:102D20000121090901EB4101A0EBC10005990870DF
:102D3000069802F0D5FF02900298013050B1FFE7EB
:102D400002980399884205D9FFE703990298401A2F
:102D5000029003E04FF0FF300290FFE7019840F24D
:102D6000A32141430398A0EBC11003900698039957
:102D700003F0A0F820B1FFE701208DF81F0040E02C
:102D80000298013078B1FFE7039902980844029055
:102D90000698029903F066F820B1FFE701208DF84C
:102DA0001F002EE00AE00698029903F05BF820B1BC
:102DB000FFE701208DF81F0023E0FFE70698019947
:102DC00002F040FE03E0009805990870FFE70498C0
:102DD00098B1FFE70598007802F016FE0599087093
:102DE0000598407802F010FE0599487005988078A3
:102DF00002F00AFE05998870FFE700208DF81F0099
:102E0000FFE79DF81F0008B080BD000080B584B0CA
:102E1000029000200190029820B9FFE701208DF870
:102E20000F0084E00298407C38B9FFE70299002047
:102E30000874029800F080F8FFE7029902204874B5
:102E4000029800F001FA38B1FFE7029904204874B3
:102E500001208DF80F006AE0029802F0ADFE38B153
:102E6000FFE702990420487401208DF80F005EE00E
:102E700002980168486820F007004860029880685E
:102E800048B1FFE746F63041C4F20001086820F07F
:102E900001000860FFE746F62C41C4F20001086813
:102EA00020F46070029A92681043086002984068AB
:102EB000013020B1FFE702984068019012E0012044
:102EC000FEF7B8FF0190019838B9FFE70299042096
:102ED000487401208DF80F0029E001980138019015
:102EE000FFE7FFE7BDF8060000F00F000299096850
:102EF0008860BDF8040002990968C860029802F071
:102F000087FE38B1FFE702990420487401208DF84C
:102F10000F000CE002990020C873029A012151733E
:102F2000029A9173029A51748DF80F00FFE79DF891
:102F30000F0004B080BD000080B582B00190019800
:102F4000006842F60001C4F20001884218D1FFE790
:102F5000FEF76AFFFFE741F21C00C4F202000168BD
:102F600041F000610160006800F00060009000988E
:102F7000FFE740F23C41C4F2422101200860FFE734
:102F800002B080BD80B588B0069005910492002003
:102F9000039002900190069818B1FFE7059820B9B8
:102FA000FFE701208DF81F00A7E0FFE70698007CEF
:102FB000012804D1FFE702208DF81F009DE006994B
:102FC00001200874FFE7FFE706990220487404987F
:102FD00068B9FFE70598C0780699C87305984078E6
:102FE00006994873059880780699887312E00598C9
:102FF000C07802F0F3FC0699C8730598407802F097
:10300000EDFC069948730598807802F0E7FC069974
:103010008873FFE70698417B827BC07B02F0B0FE9D
:10302000069908730698007B05990870069802F0C7
:1030300071FE039003984BF2C531C9F2A211A0FBB7
:103040000110C00A0190019819284AD3FFE701989E
:103050004AF6AB21CAF6AA21A0FB0110000940F2F2
:10306000A32141430398A0EBC11003900698039954
:1030700002F020FF60B1FFE7069904204874FFE7E3
:10308000069900200874FFE701208DF81F0034E046
:10309000069802F025FE02900298013000B3FFE787
:1030A0000298039988421AD2FFE7029845F28011EC
:1030B000C0F20101084402900698029902F0D2FE83
:1030C00060B1FFE7069904204874FFE706990020E5
:1030D0000874FFE701208DF81F000EE0FFE7FFE70F
:1030E000FFE7069901204874FFE70699002008745D
:1030F000FFE700208DF81F00FFE79DF81F0008B0D4
:1031000080BD000080B588B0069005910492002033
:1031100003900290069818B1FFE7059820B9FFE7E1
:1031200001208DF81F008AE0FFE70698007C012847
:1031300004D1FFE702208DF81F0080E006990120EE
:103140000874FFE7FFE7069902204874049870B9F5
:10315000FFE7059908784A7889784FF46163584306
:10316000C2EB021200EB8200084403901BE00598BA
:10317000007802F033FC4FF46161484300900598F9
:10318000407802F02BFC01460098C1EB011100EBE6
:10319000810001900598807802F020FC014601989A
:1031A00008440390FFE70698039902F083FE60B19C
:1031B000FFE7069904204874FFE706990020087489
:1031C000FFE701208DF81F0039E006980168486884
:1031D00020F005004860069802F082FD02900298F7
:1031E000013000B3FFE70298039988421AD2FFE743
:1031F000029845F28011C0F201010844029006983D
:10320000029902F02FFE60B1FFE70699042048748E
:10321000FFE7069900200874FFE701208DF81F00E2
:103220000DE0FFE7FFE7069901204874FFE70699E4
:1032300000200874FFE700208DF81F00FFE79DF8CD
:103240001F0008B080BD000080B584B0029000204F
:103250000190029820B9FFE701208DF80F0021E0CE
:1032600002980168486820F008004860FEF724FDD5
:103270000190FFE7029800684068000700280DD41D
:10328000FFE7FEF719FD0199401AB0F57A7F04D9DE
:10329000FFE703208DF80F0004E0EBE700208DF836
:1032A0000F00FFE79DF80F0004B080BD80B582B02D
:1032B0000190019802F028FE02B080BD81B000901C
:1032C00001B0704781B0009001B0704781B00090AC
:1032D00001B0704781B0009001B0704781B000909C
:1032E00001B0704785B003900291FFE7039890F812
:1032F0003C00012804D1FFE702208DF813005BE0B9
:103300000399012081F83C00FFE7FFE703990220C1
:1033100081F83D00039800684068019003980068B8
:1033200080680090019820F0700001900298016878
:10333000019808430190019803990968486003982F
:10334000006842F60041C4F20101884218D0FFE74C
:1033500003980068B0F1804F12D0FFE7039800682F
:1033600040F20041C4F20001884209D0FFE703980F
:10337000006840F60001C4F2000188420ED1FFE768
:10338000009820F08000009002984168009808435F
:1033900000900098039909688860FFE7039901206D
:1033A00081F83D00FFE70399002081F83C00FFE72A
:1033B00000208DF81300FFE79DF8130005B070475B
:1033C00080B582B00090009820B9FFE701208DF809
:1033D00007004DE0009890F83D00B0B9FFE7009974
:1033E000002081F83C00009802F0BCFE0098806C40
:1033F00038B9FFE7009943F2AD40C0F60000886499
:10340000FFE70098816C8847FFE70099022081F868
:103410003D00009951F8040B02F0FCFD00990120D9
:1034200081F84600FFE70099012081F83E000099ED
:1034300081F83F00009981F84000009981F841002F
:10344000FFE7FFE70099012081F84200009981F829
:103450004300009981F84400009981F84500FFE796
:103460000099012081F83D0000208DF80700FFE75A
:103470009DF8070002B080BD80B582B00190019830
:10348000006840F60001C4F2000188420CD1FFE759
:1034900041F21C01C4F20201086820F00400086037
:1034A0001E20FEF78BFCFFE702B080BD80B584B024
:1034B00003900398006840F60001C4F200018842BE
:1034C00019D1FFE7FFE741F21C00C4F202000168D6
:1034D00041F004010160006800F0040002900298CD
:1034E000FFE71E20019000221146FEF77BFC0198A9
:1034F000FEF76EFCFFE704B080BD000080B586B02B
:103500000490039100208DF80B00FFE7049890F8D9
:103510003C00012804D1FFE702208DF81700ABE042
:103520000499012081F83C00FFE7FFE7049902209D
:1035300081F83D000498006880680190019820F0AF
:1035400077000190019820F47F4001900198049940
:1035500009688860039800680090002872D0FFE72F
:10356000009810286ED0FFE7009820286AD0FFE767
:103570000098302866D0FFE70098402855D0FFE734
:103580000098502837D0FFE70098602840D0FFE728
:10359000009870280BD0FFE70098B0F5805F05D049
:1035A000FFE70098B0F5005F16D052E055E00498B0
:1035B0000068039B5A689968DB6802F0A3FD0498D1
:1035C000006880680190019840F0770001900198B0
:1035D00004990968886040E004980068039B5A6871
:1035E0009968DB6802F08EFD04980168886840F4F1
:1035F0008040886031E004980068039A5168D2687E
:1036000002F010FE04980068502102F095FD24E0BD
:1036100004980068039A5168D26802F02BFE04985F
:103620000068602102F088FD17E004980068039AA2
:103630005168D26802F0F6FD04980068402102F05B
:103640007BFD0AE0049800680399096802F074FDA4
:1036500003E001208DF80B00FFE70499012081F8B9
:103660003D00FFE70499002081F83C00FFE79DF84A
:103670000B008DF81700FFE79DF8170006B080BD1E
:1036800081B0009001B0704781B0009001B07047E8
:1036900081B0009001B0704781B0009001B07047D8
:1036A00081B0009001B0704781B0009001B07047C8
:1036B00081B0009001B0704780B582B00190019850
:1036C0000068006900F002010020B0EB510F2BD020
:1036D000FFE701980068C06800F002010020B0EB2D
:1036E000510F20D0FFE7019801686FF002000861D8
:1036F000019901200877019800688069800728B146
:10370000FFE70198D0F89010884708E00198D0F8BA
:10371000981088470198D0F89C108847FFE70199D6
:1037200000200877FFE7FFE701980068006900F0D4
:1037300004010020B0EB910F2CD0FFE70198006846
:10374000C06800F004010020B0EB910F21D0FFE72A
:10375000019801686FF00400086101990220087760
:1037600001980068806910F4407F05D0FFE7019858
:10377000D0F89010884708E00198D0F89810884752
:103780000198D0F89C108847FFE70199002008773E
:10379000FFE7FFE701980068006900F008010020DA
:1037A000B0EBD10F2BD0FFE701980068C06800F0A4
:1037B00008010020B0EBD10F20D0FFE7019801688D
:1037C0006FF00800086101990420087701980068EB
:1037D000C069800728B1FFE70198D0F890108847AA
:1037E00008E00198D0F8981088470198D0F89C100C
:1037F0008847FFE7019900200877FFE7FFE7019876
:103800000068006900F010010020B0EB111F2CD0FF
:10381000FFE701980068C06800F010010020B0EBDD
:10382000111F21D0FFE7019801686FF010000861B7
:1038300001990820087701980068C06910F4407F5A
:1038400005D0FFE70198D0F89010884708E001986C
:10385000D0F8981088470198D0F89C108847FFE767
:10386000019900200877FFE7FFE7019800680069E9
:10387000C00788B1FFE701980068C068C00750B171
:10388000FFE7019801686FF0010008610198D0F826
:1038900080108847FFE7FFE7019800680069C1B220
:1038A0000020B0EBD11F14D0FFE701980068C0687A
:1038B000C1B20020B0EBD11F0AD0FFE70198016828
:1038C0006FF0800008610198D0F8B0108847FFE7DA
:1038D000FFE701980068006900F040010020B0EBAC
:1038E000911F15D0FFE701980068C06800F0400103
:1038F0000020B0EB911F0AD0FFE7019801686FF03C
:10390000400008610198D0F888108847FFE7FFE77A
:1039100001980068006900F020010020B0EB511F01
:1039200015D0FFE701980068C06800F02001002072
:10393000B0EB511F0AD0FFE7019801686FF020003B
:1039400008610198D0F8A8108847FFE7FFE702B0A8
:1039500080BD000081B0009001B0704781B0009040
:1039600001B0704781B0009001B0704781B0009005
:1039700001B0704781B0009001B0704781B00090F5
:1039800001B0704781B0009001B0704781B00090E5
:1039900001B0704781B0009001B0704781B00090D5
:1039A00001B0704781B0009001B0704787B00590BA
:1039B0008DF81310039200208DF80B00039820B9A6
:1039C000FFE701208DF81B003DE1059890F83D00D0
:1039D000012840F0C380FFE79DF8130001460191E4
:1039E0001A2800F2B68001990FF2080000EB81005E
:1039F000874600BF00F034B800F036B800F038B8A1
:103A000000F03AB800F03CB800F03EB800F040B822
:103A100000F042B800F044B800F046B800F048B8F2
:103A200000F04AB800F04CB800F04EB800F050B8C2
:103A300000F053B800F056B800F059B800F05CB888
:103A400000F05FB800F062B800F065B800F068B848
:103A500000F06BB800F06EB800F071B800F074B808
:103A600003980599886478E003980599C86474E020
:103A700003980599086570E00398059948656CE01E
:103A800003980599886568E003980599C86564E01E
:103A900003980599086660E00398059948665CE01C
:103AA00003980599886658E003980599C86654E01C
:103AB00003980599086750E00398059948674CE01A
:103AC00003980599886748E003980599C86744E01A
:103AD00003980599C1F880003FE003980599C1F863
:103AE00084003AE003980599C1F8880035E003980E
:103AF0000599C1F88C0030E003980599C1F8900051
:103B00002BE003980599C1F8940026E003980599E5
:103B1000C1F8980021E003980599C1F89C001CE0C9
:103B200003980599C1F8A00017E003980599C1F81A
:103B3000A40012E003980599C1F8A8000DE00398CD
:103B40000599C1F8AC0008E003980599C1F8B000E8
:103B500003E001208DF80B00FFE76FE0059890F877
:103B60003D00002865D1FFE79DF813000146009154
:103B70000D2859D800990FF2080000EB8100874604
:103B800000F01AB800F01CB800F01EB800F020B821
:103B900000F022B800F024B800F026B800F028B8F1
:103BA00000F02AB800F02CB800F02EB800F030B8C1
:103BB00000F032B800F034B803980599886437E013
:103BC00003980599C86433E00398059908652FE0C8
:103BD0000398059948652BE003980599886527E0C7
:103BE00003980599C86523E00398059908661FE0C6
:103BF0000398059948661BE003980599886617E0C5
:103C000003980599C86613E00398059908670FE0C3
:103C10000398059948670BE003980599886707E0C2
:103C200003980599C86703E001208DF80B00FFE7B2
:103C300003E001208DF80B00FFE7FFE79DF80B0084
:103C40008DF81B00FFE79DF81B0007B070470000D0
:103C500081B0009001B0704781B0009001B0704712
:103C600084B003908DF80B1000208DF80A000398A3
:103C700090F83D00012840F01481FFE79DF80B000B
:103C8000014601911A2800F2078101990FF20800FC
:103C900000EB8100874600BF00F034B800F039B86F
:103CA00000F03EB800F043B800F048B800F04DB85E
:103CB00000F052B800F057B800F05CB800F061B8FE
:103CC00000F066B800F06BB800F070B800F075B89E
:103CD00000F07AB800F080B800F086B800F08CB838
:103CE00000F092B800F098B800F09EB800F0A4B8C8
:103CF00000F0AAB800F0B0B800F0B6B800F0BCB858
:103D000000F0C2B8039943F2AD40C0F600008864E9
:103D1000C6E0039943F27940C0F60000C864BFE0F2
:103D2000039943F2B160C0F600000865B8E003995A
:103D300043F2A960C0F600004865B1E0039943F67C
:103D40006510C0F600008865AAE0039943F65D108F
:103D5000C0F60000C865A3E0039943F68510C0F6DD
:103D6000000008669CE0039943F67D10C0F6000051
:103D7000486695E0039943F67510C0F60000886622
:103D80008EE0039943F66D10C0F60000C86687E028
:103D9000039943F28960C0F60000086780E0039948
:103DA00043F28160C0F60000486779E0039943F26E
:103DB000DD20C0F60000886772E0039943F2D52049
:103DC000C0F60000C8676BE0039943F69D10C0F68B
:103DD0000000C1F8800063E0039943F6A510C0F627
:103DE0000000C1F884005BE0039943F65140C0F63F
:103DF0000000C1F8880053E0039943F65940C0F62B
:103E00000000C1F88C004BE0039943F29960C0F6C2
:103E10000000C1F8900043E0039943F2A160C0F6AE
:103E20000000C1F894003BE0039943F65510C0F63A
:103E30000000C1F8980033E0039943F68D10C0F6F6
:103E40000000C1F89C002BE0039943F69510C0F6E2
:103E50000000C1F8A00023E0039943F29160C0F68E
:103E60000000C1F8A4001BE0039943F2C520C0F68E
:103E70000000C1F8A80013E0039943F2CD20C0F67A
:103E80000000C1F8AC000BE0039943F2BD20C0F67E
:103E90000000C1F8B00003E001208DF80A00FFE740
:103EA0009CE0039890F83D00002840F09280FFE7E6
:103EB0009DF80B00014600910D2800F285800099C5
:103EC0000FF2080000EB8100874600BF00F01AB82F
:103ED00000F01FB800F024B800F029B800F02EB8A8
:103EE00000F033B800F038B800F03DB800F042B848
:103EF00000F047B800F04CB800F051B800F056B8E8
:103F000000F05BB8039943F2AD40C0F6000088644E
:103F10005EE0039943F27940C0F60000C86457E0C0
:103F2000039943F2B160C0F60000086550E00399C0
:103F300043F2A960C0F60000486549E0039943F6E2
:103F40006510C0F60000886542E0039943F65D10F5
:103F5000C0F60000C8653BE0039943F68510C0F643
:103F60000000086634E0039943F67D10C0F60000B7
:103F700048662DE0039943F67510C0F60000886688
:103F800026E0039943F66D10C0F60000C8661FE0F6
:103F9000039943F28960C0F60000086718E00399AE
:103FA00043F28160C0F60000486711E0039943F2D4
:103FB000DD20C0F6000088670AE0039943F2D520AF
:103FC000C0F60000C86703E001208DF80A00FFE793
:103FD00003E001208DF80A00FFE7FFE79DF80A00E3
:103FE00004B07047FFE7FEE783B08DF80B009DF843
:103FF0000B0000F5FA608DF80B009DF80B10012006
:104000004BF65003C0F21E5345F62942CCF28F22E4
:1040100001FB02314FEA31114DF20B72C0F2A302E3
:104020009142019022D3FFE79DF80B1000208907F1
:104030000090C1B9FFE79DF80B004BF65002C0F2AB
:104040001E5245F62941CCF28F2100FB01204FEA98
:10405000B00145F62842C0F28F220020914288BF6D
:1040600001200090FFE700980190FFE7019800F021
:10407000010003B07047000080B582B040F6E00058
:10408000C2F20000019046F20041C4F2000101605A
:104090000821416000228260C2604FF4402101612A
:1040A0004FF4801141610276012141768276C27619
:1040B00002774177FCF79EFF18B1FFE7FCF72AFA79
:1040C000FFE702B080BD000080B586B000200590FB
:1040D000049003900290FFE741F21800C4F202003E
:1040E000016841F004010160006800F004000190E3
:1040F0000198FFE74FF48070029002200390059032
:1041000040F60000C4F2010002A9FDF745FC06B02C
:1041100080BD000080B582B000208DF80600ADF8AB
:104120000400009040F64410C2F2000042F6000184
:10413000C4F2000101604FF0FF3141604FF4807123
:104140008160FEF763FE18B1FFE7FCF7E3F9FFE7D4
:1041500000208DF804008DF805008DF8060040F66B
:104160004410C2F2000001A90122FEF7CBFF18B1F2
:10417000FFE7FCF7CFF9FFE701228DF800208DF86B
:1041800001208DF8022000208DF8030040F6441035
:10419000C2F200006946FEF7F5FE18B1FFE7FCF732
:1041A000B9F9FFE702B080BD80B588B00021019168
:1041B00007910691059104910391029140F65810E0
:1041C000C2F2000040F60002C4F2000202604FF6A4
:1041D000FF12426081604FF47A72C26001618161B6
:1041E000FFF7EEF818B1FFE7FCF794F9FFE74FF49B
:1041F0008050049040F65810C2F2000004A9FFF766
:104200007DF918B1FFE7FCF785F9FFE70020029080
:10421000039040F65810C2F2000002A9FFF762F8BE
:1042200018B1FFE7FCF776F9FFE708B080BD0000A2
:10423000FFE7FEE7FFE7FEE788B0079006910592EB
:10424000079800F0070004900498C0F107000528C3
:1042500003D3FFE70420019004E00498C0F10700B5
:104260000190FFE70198039004980430062803D8D2
:10427000FFE70020009003E0049803380090FFE778
:104280000098029006980399012202FA01F101397F
:104290000840029B984005999A40013A1140084312
:1042A00008B0704780B58AB0DDF830C0CDF820C0C6
:1042B0000793069205910490BDF814000390BDF891
:1042C0000C00000B01460291042855D802990FF208
:1042D000080000EB8100874600F008B800F014B831
:1042E00000F020B800F02CB800F038B80498059918
:1042F000069A079BDDF820C0EE46CEF800C000F01D
:1043000001FF8DF827003BE004980599069A079B6A
:10431000DDF820C0EE46CEF800C000F0A3FD8DF819
:1043200027002DE004980599069A079BDDF820C028
:10433000EE46CEF800C000F05FFE8DF827001FE0CB
:1043400004980599069A079BDDF820C0EE46CEF842
:1043500000C000F001FD8DF8270011E004980599D8
:10436000069A079BDDF820C0EE46CEF800C000F0AC
:10437000BDFD8DF8270003E001208DF82700FFE741
:104380009DF827000AB080BD80B58AB0DDF830C046
:10439000CDF820C00793069205910490BDF8140053
:1043A0000390BDF80C0000090146029103283FD894
:1043B00002990FF2080000EB8100874600F006B872
:1043C00000F012B800F01CB800F026B80498059967
:1043D000069A079BDDF820C0EE46CEF800C000F03C
:1043E00099FF8DF827002BE004980599069A079B02
:1043F000DDF820C0EE46CEF800C000F0C3FE1BE0A2
:1044000004980599069A079BDDF820C0EE46CEF881
:1044100000C000F0CFFE0FE004980599069A079BB4
:10442000DDF820C0EE46CEF800C000F013FF03E038
:1044300001208DF8270003E000208DF82700FFE71A
:104440009DF827000AB080BD80B58EB08DF837008A
:104450000C910B929DF837000690002107910120E6
:104460000890059109900E200A900C98C0F34F30E7
:1044700001900C98C000043080B202900B98C0F3F9
:104480004F3003900B98C000043080B2049040F687
:10449000D400C2F20000006801A9FCF719F918B1B4
:1044A000FFE7FCF737F8FFE70EB080BD80B582B0BC
:1044B0008DF807009DF80710481E009102280DD3C3
:1044C000FFE70098032812D1FFE740F6DC00C2F2B4
:1044D000000000680E21FFF7C3FBFFE740F6D400A1
:1044E000C2F2000000680621FDF79EF8FFE702B067
:1044F00080BD000080B58AB0DDF830C0CDF820C0A6
:104500000793069205910490BDF814000390BDF83E
:104510000C00000B01460291062867D802990FF2A1
:10452000080000EB8100874600F00CB800F016B8D8
:1045300000F020B800F02AB800F034B800F03EB81F
:1045400000F048B804980599069A079BDDF820C04A
:10455000EE46CEF800C000F04BFF4BE00498059902
:10456000069A079BDDF820C0EE46CEF800C000F0AA
:1045700091FF3FE004980599069A079BDDF820C05B
:10458000EE46CEF800C000F04FFF33E004980599E6
:10459000069A079BDDF820C0EE46CEF800C000F07A
:1045A00051FF27E004980599069A079BDDF820C083
:1045B000EE46CEF800C000F061FF1BE004980599BC
:1045C000069A079BDDF820C0EE46CEF800C000F04A
:1045D0001DFF0FE004980599069A079BDDF820C09F
:1045E000EE46CEF800C000F03BFF03E001208DF85E
:1045F000270003E000208DF82700FFE79DF8270043
:104600000AB080BD80B586B04FF0126005904FF0C3
:104610007F600490002003904FF47021029101917B
:1046200000910599049AFFF70FFF0399029A012060
:10463000FFF70AFF0199009A0220FFF705FF06B075
:1046400080BD000080B586B00490039102920020E6
:1046500001900498E8B1FFE7049940F6D400C2F253
:1046600000000160006845F6C902C0F6000206219C
:10467000FCF7A8FE8DF803009DF8030040B1FFE7AA
:104680009DF80400FFF712FF02208DF8170059E093
:1046900007E09DF80400FFF709FF01208DF81700DF
:1046A00050E0019801300190039838B1FFE703987A
:1046B00040F6D801C2F20001086007E09DF804004E
:1046C000FFF7F4FE02208DF817003BE0019801305F
:1046D00001900298E8B1FFE7029940F6DC00C2F2CF
:1046E00000000160006845F2F572C0F600020E217C
:1046F000FFF75CF98DF802009DF8020040B1FFE77A
:104700009DF80400FFF7D2FE02208DF8170019E093
:1047100007E09DF80400FFF7C9FE04208DF817009C
:1047200010E0019801300190FFF76CFF40F2C801E2
:10473000C2F20001087840F00100087000208DF8F6
:104740001700FFE79DF8170006B080BD80B588B060
:10475000079800F0604007909DF81F0040F010009F
:104760008DF81F009DF81F0040F008008DF81F0015
:104770009DF81E0000F0F00003308DF81E0049F691
:10478000F120ADF80C004AF6BF70C5F278600290D7
:104790004AF6CD30C1F23420019001A805900520E1
:1047A0000690FA20ADF81000FFE7FBF7A3FD002804
:1047B00000F06781FFE740F20000C2F200000078DD
:1047C00000EB800140F60C20C2F2000000EB8100FB
:1047D000807900F00F0002281DD1FFE740F20000B1
:1047E000C2F20000007800EB800140F60C20C2F21B
:1047F000000000EB810C50F82100DCF80410DCF81C
:104800000820DCF80C30DCF810C0EE46CEF800C012
:10481000FFF748FD2BE140F20000C2F200000078F3
:1048200000EB800140F60C20C2F2000000EB81009A
:1048300080790007E8B9FFE740F20000C2F200000B
:10484000007800EB800140F60C20C2F2000000EB83
:10485000810C50F82100DCF80410DCF80820DCF8AA
:104860000C30DCF810C0EE46CEF800C0FFF78CFD2F
:10487000FCE040F20000C2F20000007800EB800192
:1048800040F60C20C2F2000000EB8100807900F0BD
:104890000F0001281DD1FFE740F20000C2F2000026
:1048A000007800EB800140F60C20C2F2000000EB23
:1048B000810C50F82100DCF80410DCF80820DCF84A
:1048C0000C30DCF810C0EE46CEF800C0FFF712FE48
:1048D000CBE040F20000C2F20000007800EB800163
:1048E00040F60C20C2F2000000EB8100807900F05D
:1048F0000F0003281DD1FFE740F20000C2F20000C4
:10490000007800EB800140F60C20C2F2000000EBC2
:10491000810C50F82100DCF80410DCF80820DCF8E9
:104920000C30DCF810C0EE46CEF800C000F0C0FD40
:104930009AE040F20000C2F20000007800EB800133
:1049400040F60C20C2F2000000EB8100807900F0FC
:104950000F00042839D0FFE740F20000C2F2000047
:10496000007800EB800140F60C20C2F2000000EB62
:104970008100807900F00F00052826D0FFE740F283
:104980000000C2F20000007800EB800140F60C202D
:10499000C2F2000000EB8100807900F00F000628D1
:1049A00013D0FFE740F20000C2F20000007800EBF5
:1049B000800140F60C20C2F2000000EB81008079FB
:1049C00000F00F0007281DD1FFE740F20000C2F2FF
:1049D0000000007800EB800140F60C20C2F20000DD
:1049E00000EB810C50F82100DCF80410DCF8082002
:1049F000DCF80C30DCF810C0EE46CEF800C000F059
:104A000047F830E040F20000C2F20000007800EB0E
:104A1000800140F60C20C2F2000000EB810080799A
:104A200000F00F0008281DD1FFE740F20000C2F29D
:104A30000000007800EB800140F60C20C2F200007C
:104A400000EB810C50F82100DCF80410DCF80820A1
:104A5000DCF80C30DCF810C0EE46CEF800C0FBF7F6
:104A60001BFDFFE7FFE7FFE7FFE7FFE7FFE740F298
:104A70000001C2F200010878013000F07F000870E8
:104A8000FFE707980499059A069B00F0B5F88CE6B5
:104A900080B588B0DDF828C0CDF818C00593049221
:104AA000039102909DF80E0000F00F0004380146BB
:104AB0000191032846D801990FF2080000EB81000C
:104AC000874600BF00F006B800F012B800F01EB82C
:104AD00000F02AB802980399049A059BDDF818C0E3
:104AE000EE46CEF800C000F04FFD8DF81F002DE01F
:104AF00002980399049A059BDDF818C0EE46CEF89B
:104B000000C000F08DFD8DF81F001FE00298039992
:104B1000049A059BDDF818C0EE46CEF800C000F000
:104B2000CDFD8DF81F0011E002980399049A059BB2
:104B3000DDF818C0EE46CEF800C000F00DFE8DF88E
:104B40001F0003E001208DF81F00FFE79DF81F0004
:104B500008B080BD80B584B0039040F6D800C2F2A2
:104B6000000001680A68516841F01001516000229C
:104B70008DF80A20ADF808200192039909788DF884
:104B80000810039949788DF80910039989788DF8F0
:104B90000A10006802A9FEF7B5FA18B1FFE7FBF7A3
:104BA000B9FCFFE70398C0788DF8070003980079F7
:104BB0008DF80500039840798DF8060003988079F8
:104BC0008DF8040040F6D800C2F20000006801A988
:104BD0000022FEF7D7F918B1FFE7FBF79BFCFFE7D0
:104BE00040F6D800C2F2000000680168486820F072
:104BF0001000486004B080BD80B586B00490039377
:104C0000029201919DF8120000F00F0003280BD1D1
:104C1000FFE7BDF80410029A9DF80C30049800F0EC
:104C20000BF88DF8170003E001208DF81700FFE75F
:104C30009DF8170006B080BD80B594B01290ADF815
:104C4000461010928DF83F300020089004210B91FF
:104C50008DF838000C90129A059962F31C010591A9
:104C60009DF83F108DF813108DF81200FFE79DF8A6
:104C70001300012865DBFFE79DF81300052803DB1F
:104C8000FFE70420019003E09DF813000190FFE787
:104C900001988DF81100BDF846009DF812100844E7
:104CA000ADF81400059820F060400A909DF81100BE
:104CB00040000D9000200390FFE703989DF811102D
:104CC00088421ADAFFE710989DF81210039A1144EF
:104CD00030F8110006A901EB4202507010989DF8BF
:104CE0001230039A134400EB4300407801F812009D
:104CF000FFE7039801300390DFE740F6D400C2F2EB
:104D00000000006809A906AA08ABFBF735FC8DF87E
:104D10000B009DF80B0028B1FFE79DF80B008DF804
:104D20004F0012E09DF811109DF81300401A8DF805
:104D300013009DF811109DF8120008448DF8120020
:104D400095E700208DF84F00FFE79DF84F0014B065
:104D500080BD00007047000080B590B0DDF848C00D
:104D6000CDF83CC00E930D920C910B900020049056
:104D7000042107918DF8280008900C99019861F39F
:104D80001C0001909DF8070040F008008DF8070016
:104D9000019820F06040069006200990BDF8300090
:104DA000009049208DF8080053208DF80900BDF8C7
:104DB00000006FF31F3044F6D351C1F26201A0FB33
:104DC00001012F2000EB91108DF80A00BDF80000C2
:104DD0006FF31F3048F21F51C5F2EB11A0FB011019
:104DE000400946F26761C6F2666180FB012303F069
:104DF0001C0202EB9302A0EB42002F308DF80B0057
:104E0000BDF800006FF31F304CF6CD42CCF6CC421B
:104E1000A0FB0230C00880FB011303F0FC0101EB92
:104E20009301A0EB41002F308DF80C00BDF800007D
:104E300001466FF31F31A1FB0221C90801EB81017B
:104E4000A0EB41002F308DF80D0040F6D400C2F2E7
:104E50000000006805A902AA04ABFBF78DFB10B0A7
:104E600080BD000080B590B0DDF848C0CDF83CC0F2
:104E70000E930D920C910B90002004900421079149
:104E80008DF8280008900C99019861F31C0001909E
:104E90009DF8070040F008008DF80700019820F009
:104EA000604006900720099055208DF80800532097
:104EB0008DF8090054208DF80A0041208DF80B0070
:104EC00056208DF80C004B208DF80D0049208DF8F0
:104ED0000E0040F6D400C2F20000006805A902AA44
:104EE00004ABFBF749FB10B080BD000080B590B06B
:104EF000DDF848C0CDF83CC00E930D920C910B909C
:104F000000200490042107918DF8280008900C9946
:104F1000019861F31C0001909DF8070040F0080023
:104F20008DF80700019820F0604006900620099057
:104F3000BDF83000009054208DF8080053208DF803
:104F40000900BDF800006FF31F3044F6D351C1F2E1
:104F50006201A0FB01012F2000EB91108DF80A00E7
:104F6000BDF800006FF31F3048F21F51C5F2EB117E
:104F7000A0FB0110400946F26761C6F2666180FB42
:104F8000012303F01C0202EB9302A0EB42002F303E
:104F90008DF80B00BDF800006FF31F304CF6CD42CA
:104FA000CCF6CC42A0FB0230C00880FB011303F01A
:104FB000FC0101EB9301A0EB41002F308DF80C00B8
:104FC000BDF8000001466FF31F31A1FB0221C908A3
:104FD00001EB8101A0EB41002F308DF80D0040F670
:104FE000D400C2F20000006805A902AA04ABFBF7D6
:104FF000C3FA10B080BD000080B590B0DDF848C0A5
:10500000CDF83CC00E930D920C910B9000200490B3
:10501000042107918DF8280008900C99019861F3FC
:105020001C0001909DF8070040F008008DF8070073
:10503000019820F06040069006200990BDF83000ED
:10504000009055208DF8080053208DF80900BDF818
:1050500000006FF31F3044F6D351C1F26201A0FB90
:1050600001012F2000EB91108DF80A00BDF800001F
:105070006FF31F3048F21F51C5F2EB11A0FB011076
:10508000400946F26761C6F2666180FB012303F0C6
:105090001C0202EB9302A0EB42002F308DF80B00B4
:1050A000BDF800006FF31F304CF6CD42CCF6CC4279
:1050B000A0FB0230C00880FB011303F0FC0101EBF0
:1050C0009301A0EB41002F308DF80C00BDF80000DB
:1050D00001466FF31F31A1FB0221C90801EB8101D9
:1050E000A0EB41002F308DF80D0040F6D400C2F245
:1050F0000000006805A902AA04ABFBF73DFA10B056
:1051000080BD000080B590B0DDF848C0CDF83CC04F
:105110000E930D920C910B900020049004210791A6
:105120008DF8280008900C99019861F31C000190FB
:105130009DF8070040F008008DF80700019820F066
:10514000604006900620099055208DF808004E20FA
:105150008DF8090049208DF80A0056208DF80B00C3
:1051600045208DF80C0052208DF80D0040F6D4003B
:10517000C2F20000006805A902AA04ABFBF7FCF923
:1051800010B080BD80B585B0DDF81CC0CDF810C072
:10519000039302920191009040F2C801C2F2000113
:1051A00008780122824300F0FE00104408700020BD
:1051B00005B080BD80B58CB0DDF838C0CDF828C012
:1051C0000993089207910690BDF8200020B9FFE7E7
:1051D00001208DF82F0039E0BDF81C000590BDF8C6
:1051E000140000F00F00BDF82010CA000221B1FB2E
:1051F000F2F1884226D1FFE700200390029001904F
:10520000FFE70198BDF82010884213DAFFE7019903
:1052100006A80844807AC90000FA01F202990398AE
:10522000891840EBE27002910390FFE7019801308A
:105230000190E6E702988008C00710B1FFE701F08F
:1052400039F9FFE700208DF82F00FFE79DF82F00C8
:105250000CB080BD80B5A0B0DDF888C0CDF878C0B6
:105260001D931C921B911A90BDF87000082804DB56
:10527000FFE701208DF87F0048E046F24451C0F678
:10528000000102A86022FAF79FFF9DF8720017281C
:105290002EDCFFE79DF873003B2829DCFFE79DF833
:1052A00074003B2824DCFFE79DF8750063281FDCB1
:1052B000FFE79DF876000C281ADCFFE79DF87500E3
:1052C0009DF877100191FEF78FFE0146019801EBE2
:1052D000410202A901EB02119DF8762051F822103B
:1052E000884205DCFFE79DF87800072804DBFFE72C
:1052F00001208DF87F0009E01AA80A30FFF72AFC88
:10530000FFE7FFE700208DF87F00FFE79DF87F00B3
:1053100020B080BD80B594B0DDF858C0CDF84CC049
:105320001293119210910F90002201920892042082
:105330000B9007200D908DF838200C92109905984D
:1053400061F31C0005909DF8170040F008008DF8EF
:1053500017009DF8170000F0F80001308DF81700D5
:105360009DF81600022161F31F108DF816000598B4
:1053700020F060400A908DF81220ADF8102040F621
:10538000D800C2F200000290006804A9FDF764FC96
:10539000019A02989DF810108DF818109DF81110C0
:1053A0008DF819109DF812108DF81A1003920068EC
:1053B00003A9FDF703FC9DF80F008DF81B009DF875
:1053C0000D008DF81C009DF80E008DF81D009DF855
:1053D0000C008DF81E0040F6D400C2F200000068F8
:1053E00009A906AA08ABFBF7C7F814B080BD0000F6
:1053F00080B585B0DDF81CC0CDF810C003930292D3
:1054000001910090002005B080BD000080B585B0FE
:10541000DDF81CC0CDF810C00393029201910090FA
:10542000002005B080BD000080B585B0DDF81CC04F
:10543000CDF810C00393029201910090002005B0B6
:1054400080BD000080B585B0DDF81CC0CDF810C06F
:105450000393029201910090002005B080BD0000EE
:1054600080B585B0DDF81CC0CDF810C00393029262
:1054700001910090002005B080BD000080B586B08D
:10548000DDF820C0CDF814C004930392029101907E
:1054900001F010F880B585B0DDF81CC0CDF810C063
:1054A0000393029201910090002005B080BD00009E
:1054B00080B592B0DDF850C0CDF844C010930F9283
:1054C0000E910D9000200690042109918DF8300076
:1054D0000A900E9A039962F31C0103919DF80F1034
:1054E00041F008018DF80F10039921F060410891F7
:1054F00008210B9147218DF8101041218DF81110D2
:1055000053218DF812102D218DF813100290FFE712
:10551000029803282CDCFFE7BDF83800029A0C2122
:10552000A1EB8201C84000F00F00019001980A2809
:1055300012D3FFE701984CF6CD41CCF6CC41A0FB4D
:105540000121C90801EB8101A0EB41004130029922
:1055500004AA1144087106E001983030029904AAA7
:1055600011440871FFE7FFE7029801300290CFE78E
:1055700040F6D400C2F20000006807A904AA06ABF6
:10558000FAF7FAFF12B080BD80B590B0DDF848C0E0
:10559000CDF83CC00E930D920C910B90002004901E
:1055A000042107918DF8280008900C99019861F367
:1055B0001C0001909DF8070040F008008DF80700DE
:1055C000019820F06040069008200990BDF8300056
:1055D00000904D208DF8080043208DF8090020210F
:1055E0008DF80A1053228DF80B20BDF80020120907
:1055F0008DF80C208DF80D108DF80E009DF8000030
:1056000000F00F008DF80F0040F6D400C2F2000049
:10561000006805A902AA04ABFAF7AEFF10B080BD7E
:1056200080B590B0DDF848C0CDF83CC00E930D9227
:105630000C910B9000200490042107918DF8280014
:1056400008900C99019861F31C0001909DF80700E7
:1056500040F008008DF80700019820F060400690A7
:1056600008200990BDF8300000904D208DF808000A
:1056700044208DF8090020208DF80A0053218DF870
:105680000B10BDF8001009098DF80C108DF80D00F5
:1056900043208DF80E009DF8000000F00F008DF8FB
:1056A0000F0040F6D400C2F20000006805A902AA6B
:1056B00004ABFAF761FF10B080BD000080B590B078
:1056C000DDF848C0CDF83CC00E930D920C910B90C4
:1056D00000200490042107918DF8280008900C996F
:1056E000019861F31C0001909DF8070040F008004C
:1056F0008DF80700019820F060400690082009907E
:10570000BDF8300000904D208DF8080048208DF83D
:10571000090020208DF80A0053218DF80B10BDF8E8
:10572000001009098DF80C108DF80D0043208DF83C
:105730000E009DF8000000F00F008DF80F0040F6FD
:10574000D400C2F20000006805A902AA04ABFAF76F
:1057500013FF10B080BD000080B590B0DDF848C0E8
:10576000CDF83CC00E930D920C910B90002004904C
:10577000042107918DF8280008900C99019861F395
:105780001C0001909DF8070040F008008DF807000C
:10579000019820F06040069008200990BDF8300084
:1057A00000904D208DF8080049208DF80900202038
:1057B0008DF80A0053218DF80B10BDF8001009096F
:1057C0008DF80C108DF80D0043208DF80E009DF81B
:1057D000000000F00F008DF80F0040F6D400C2F278
:1057E0000000006805A902AA04ABFAF7C5FE10B0D4
:1057F00080BD000080B58CB00B9040F2C800C2F2B2
:1058000000000078C00700285CD0FFE7002004906B
:10581000039901F0604103919DF80F1041F01001D0
:105820008DF80F109DF80F1041F008018DF80F1042
:105830009DF80F1001F0F80101318DF80F109DF85F
:105840000E10022262F31F118DF80E109DF80E103B
:1058500041F00F018DF80E10ADF80C00039921F006
:1058600060410691042107918DF8280008900120DD
:10587000099040F6D000C2F20000016801310160D9
:10588000039921F0604100910068B0F5807F07D353
:10589000FFE740F6D001C2F2000100200860FFE7F8
:1058A00040F6D000C2F2000000688DF8040040F617
:1058B000D400C2F20000006805A901AA04ABFAF7FF
:1058C0005BFEFFE70CB080BD80B58EB00D90FFE7AA
:1058D0000D98002106AA04ABFBF788F800285CD1DC
:1058E000FFE70898042857D1FFE740F6CC00C2F242
:1058F0000000007840F20001C2F200010978401A6D
:1059000081300006002801D4FFE746E040F6CC00D5
:10591000C2F200000078013000F07F00ADF80E0008
:105920000799029861F31C0002909DF80A0000F0AC
:105930000F000F2820D1FFE79DF80A109DF80B00FB
:1059400000F0070240F2CC00C2F2000000EB02229D
:1059500001F0F003D15C41F00101D1549DF80A102F
:105960009DF80B2002F0070200EB022001F0F0018D
:1059700001440020886010E00899099A0A9BBDF84C
:105980000EC00298EE46CEF804C00DF1100CCEF811
:1059900000C000F099FCFFE79AE70EB080BD000060
:1059A00082B00190019840F20401C2F2000109683E
:1059B000C90844F6D352C1F26202A1FB022189094F
:1059C00048430090FFE700BFFFE70098411E0091A9
:1059D0000028F8D1FFE702B07047000082B08DF8D0
:1059E0000700002000909DF80700000900EB8000F0
:1059F0004000009000989DF8071001F00F01084446
:105A0000C0B202B07047000082B08DF807000020DD
:105A10000090FFE79DF807000A2809D3FFE70098E8
:105A2000013000909DF807000A388DF80700F1E773
:105A3000009800F00F019DF8070040EA011002B045
:105A40007047000080B586B0059004910020039057
:105A50000290019000900599C97B03910599497BBB
:105A600002910599897B01910090FFE700980499C4
:105A7000884280F08C80FFE70298012818D0FFE769
:105A80000298032814D0FFE70298052810D0FFE7FA
:105A9000029807280CD0FFE70298082808D0FFE7F3
:105AA00002980A2804D0FFE702980C281BD1FFE7D0
:105AB00001981E2804D8FFE701980130019011E0F9
:105AC00002980C2806D0FFE70298013002900120CE
:105AD000019006E0012002900190039801300390AC
:105AE000FFE7FFE74EE0029804280CD0FFE702989A
:105AF000062808D0FFE70298092804D0FFE702989B
:105B00000B280FD1FFE701981D2804D8FFE7019863
:105B10000130019005E002980130029001200190CF
:105B2000FFE72EE0029802282AD1FFE701981B2800
:105B300004D8FFE701980130019020E001981C286B
:105B400011D1FFE7BDF80C0000F08EF820B1FFE79F
:105B500001980130019005E0029801300290012087
:105B60000190FFE70AE001981D2806D1FFE702989F
:105B70000130029001200190FFE7FFE7FFE7FFE718
:105B8000FFE7FFE7FFE70098013000906EE703981A
:105B90000599C87302980599487301980599887307
:105BA00003989DF808109DF8042000F0E9F8059985
:105BB000087306B080BD000080B584B0029000205C
:105BC0000190FCF779F80190FFE7029800684068BF
:105BD000800600280DD4FFE7FCF76EF80199401A03
:105BE000B0F57A7F04D9FFE703208DF80F000AE0B3
:105BF000EBE702980168486840F010004860002018
:105C00008DF80F00FFE79DF80F0004B080BD000085
:105C100080B584B002900020019002980168486825
:105C200020F010004860FCF747F80190FFE7029869
:105C300000684068800600280DD4FFE7FCF73CF8B8
:105C40000199401AB0F57A7F04D9FFE703208DF857
:105C50000F0004E0EBE700208DF80F00FFE79DF850
:105C60000F0004B080BD000081B0ADF80000BDF8A9
:105C70000000800720B1FFE700208DF803002BE033
:105C8000BDF8000045F62941CCF28F2148434FEA88
:105C9000B00045F62941C0F28F21884204D3FFE7C6
:105CA00001208DF8030017E0BDF8000045F62941FA
:105CB000CCF28F2148434FEA30104DF20A71C0F206
:105CC000A301884204D8FFE701208DF8030003E018
:105CD00000208DF80300FFE79DF8030001B0704736
:105CE00082B001900020ADF80200ADF800000198EC
:105CF0000068006AADF8020001980068406AADF8DB
:105D00000000BDF80210BDF8000040EA014002B0FA
:105D10007047000084B003900020ADF80A00ADF891
:105D20000800ADF806000090039800688069ADF89F
:105D30000A0003980068C069ADF80600039800687F
:105D40008069ADF80800BDF80A00BDF80810884267
:105D50000AD0FFE7BDF8081003980068C06980B258
:105D600040EA0140009007E0BDF80A10BDF80600C7
:105D700040EA01400090FFE7009804B0704700003F
:105D800084B003908DF80B108DF80A20002001904C
:105D90000090039800F5FA6001909DF80B0002282E
:105DA0002ED8FFE79DF80B001721484348F63961CC
:105DB000C3F6E301A0FB01019DF80A0000EB5100CE
:105DC00001990844013900EB910048F21F52C5F2D5
:105DD000EB12A1FB0221A0EB511000EBD11004301B
:105DE00044F62511C2F29241A0FB0121421A01EBB7
:105DF00052029108C900A1EB9201401A00902CE0D8
:105E00009DF80B001721484348F63961C3F6E301BA
:105E1000A0FB01019DF80A0000EB51000199084424
:105E200000EB910048F21F52C5F2EB12A1FB0221D8
:105E3000A0EB511000EBD110023044F62511C2F254
:105E40009241A0FB0121421A01EB52029108C900C4
:105E5000A1EB9201401A0090FFE79DF8000004B00A
:105E60007047000080B584B00390029100208DF847
:105E700007000398FFF7A0FE20B1FFE701208DF88F
:105E8000070013E0BDF80A00039909680862BDF82D
:105E900008000399096848620398FFF7B9FE20B12A
:105EA000FFE701208DF80700FFE7FFE79DF80700F7
:105EB00004B080BD80B584B00390029100208DF8BD
:105EC00007000398FFF778FE20B1FFE701208DF867
:105ED000070013E0BDF80A00039909688861BDF85E
:105EE000080003990968C8610398FFF791FE20B183
:105EF000FFE701208DF80700FFE7FFE79DF80700A7
:105F000004B080BD7047000080B582B0009000985A
:105F10000138B0F1807F03D3FFE70120019019E041
:105F2000009801384EF21401CEF2000108604FF0E3
:105F3000FF300F2100F07EFA4EF21801CEF2000180
:105F4000002008604EF21002CEF20002072111601C
:105F50000190FFE7019802B080BD000080B5FBF71B
:105F6000B1FE80BD80B596B00CA801902821FAF74B
:105F70005DF90198002102910B910A910991089114
:105F8000079106910591049103910A220C92012236
:105F900010921023119312920222139214914FF433
:105FA00060111591FCF7CCFA18B1FFE7FAF7B2FAD5
:105FB000FFE70F20079002210891002009904FF47D
:105FC00080620A920B9007A8FCF7E4F818B1FFE78B
:105FD000FAF7A0FAFFE7012003904FF40070049055
:105FE00003A8FBF7F3FF18B1FFE7FAF793FAFFE70F
:105FF0004FF0E06100221046FCF76EFA16B080BD4B
:106000007047000080B540F65810C2F20000FDF75E
:1060100053FB80BD83B0029001910298006800900C
:10602000029842F60041C4F20101884215D0FFE710
:106030000298B0F1804F10D0FFE7029840F2004183
:10604000C4F20001884208D0FFE7029840F6000140
:10605000C4F2000188420AD1FFE7009820F07000E6
:10606000009001984168009808430090FFE702986B
:1060700042F60041C4F20101884215D0FFE70298C0
:10608000B0F1804F10D0FFE7029840F20041C4F217
:106090000001884208D0FFE7029840F60001C4F2F0
:1060A000000188420AD1FFE7009820F44070009078
:1060B0000198C168009808430090FFE7009820F01D
:1060C000800001994969084300900098029908608E
:1060D000019880680299C8620198006802998862F4
:1060E000029842F60041C4F20101884205D1FFE75F
:1060F0000198006902990863FFE70299012048614D
:1061000003B0704785B00490039102920193049804
:1061100080680090009820F47F40009003980299D6
:10612000019A41EA02210143009808430090009837
:106130000499886005B0704783B00290019102987D
:1061400080680090009820F07000009001980099FD
:10615000084340F00700009000980299886003B05F
:106160007047000081B00090009943F69D10C0F682
:106170000000C1F88000009943F6A510C0F60000A9
:10618000C1F88400009943F65140C0F60000C1F800
:106190008800009943F65940C0F60000C1F88C0011
:1061A000009943F29960C0F60000C1F89000009990
:1061B00043F2A160C0F60000C1F89400009943F6D4
:1061C0005510C0F60000C1F89800009943F68D10F4
:1061D000C0F60000C1F89C00009943F69510C0F687
:1061E0000000C1F8A000009943F29160C0F60000E1
:1061F000C1F8A400009943F2C520C0F60000C1F820
:10620000A800009943F2CD20C0F60000C1F8AC0010
:10621000009943F2BD20C0F60000C1F8B00001B003
:106220007047000085B00490039102920498006AC0
:1062300000900499086A20F00100086204988069BF
:106240000190019820F0F00001900299019840EA35
:1062500001100190009820F00A0000900399009826
:106260000843009001980499886100980499086295
:1062700005B0704785B00490039102920498006ABB
:1062800000900499086A20F0100008620498806960
:106290000190019820F4704001900299019840EA21
:1062A00001300190009820F0A00000900399009820
:1062B00040EA0110009001980499886100980499BF
:1062C000086205B07047000080B586B08446099822
:1062D000DDF820E0CDF814C0049103920293ADF8EC
:1062E0000600059BBDF8060000EB800040F60C217F
:1062F000C2F2000101EB8002506863F31C005060A1
:106300009DF81030BDF8060000EB800211F8220065
:1063100003F0010300F0FE00184401F822009DF88C
:106320000C30BDF8060000EB800211F8220003F0EB
:10633000010300F0FD0040EA430001F8220002984A
:10634000BDF8062002EB820201EB820108810020E9
:106350000090FFE700980299884214D2FFE708985E
:10636000009A805CBDF8061001EB810340F60C2119
:10637000C2F2000101EB830111448872FFE700982B
:1063800001300090E6E79DF8060040F6CC01C2F22D
:106390000001087006B080BD80B540F6E000C2F292
:1063A0000000FAF72DFC80BD80B540F6E000C2F297
:1063B0000000FAF725FC80BDFFE7FEE781B08DF80D
:1063C00003009DF90300002812D4FFE79DF9031094
:1063D00001F01F02012090404A094EF28011CEF2D6
:1063E000000141F82200BFF34F8FBFF36F8FFFE72B
:1063F00001B0704781B08DF803009DF903000028BB
:106400000ED4FFE79DF9031001F01F020120904018
:106410004A094EF20011CEF2000141F82200FFE7D6
:1064200001B070474EF60C50CEF200000068C0F389
:106430000220704782B08DF8070000919DF9070097
:1064400000280AD4FFE7009800019DF907104EF2DA
:106450000042CEF2000288540BE0009800019DF843
:10646000071001F00F014EF61452CEF200028854CC
:10647000FFE702B07047000083B00290029800F07E
:10648000070000904EF60C51CEF200010868019012
:1064900001984FF6FF02104001900198009A40EADF
:1064A00002200022C0F2FA521043019001980860C5
:1064B00003B07047BFF34F8F4EF60C51CEF2000180
:1064C000086800F4E0600422C0F2FA521043086049
:1064D000BFF34F8FFFE700BFFDE7000080B582B03C
:1064E00000200190FFF73EFDFBF7FAFBFFF73AFDB6
:1064F000FDF7EAFDFDF7C0FDFDF70CFEFDF754FECC
:1065000040F6E000C2F2000040F64411C2F2000181
:1065100040F65812C2F20002FEF794F878B9FFE78D
:1065200040F6E000C2F200000090FBF71FF8009870
:1065300048F60241F9F7F6FFFEF708F9FFE7FFE733
:10654000FEE700001F0000001C0000001F0000000C
:106550001E0000001F0000001E0000001F000000C1
:106560001F0000001E0000001F0000001E000000B1
:106570001F0000001F0000001D0000001F000000A1
:106580001E0000001F0000001E0000001F00000091
:106590001F0000001E0000001F0000001E00000081
:1065A0001F000000000000000000000001020304C2
:1065B00006070809000000000102030402030405A5
:1065C000060708090A0B0C0D0E0F1010010202033A
:1065D0000405060708090A0B0C0D0E0F1010010226
:1065E00000660008000000201000000028010008DC
:1065F0001066000810000020001A00004401000886
:10660000010000000024F400010000001000000060
:04000005080000ED02
:00000001FF
